BL51 BANKED LINKER/LOCATER V5.11                                                        02/09/2014  15:07:21  PAGE 1


BL51 BANKED LINKER/LOCATER V5.11, INVOKED BY:
D:\PROGRAM FILES\KEIL\C51\BIN\BL51.EXE STARTUP.obj, 发送文件.obj TO 485_Send


MEMORY MODEL: SMALL


INPUT MODULES INCLUDED:
  STARTUP.obj (?C_STARTUP)
  发送文件.obj (穇送文件)


LINK MAP OF MODULE:  485_Send (?C_STARTUP)


            TYPE    BASE      LENGTH    RELOCATION   SEGMENT NAME
            -----------------------------------------------------

            * * * * * * *   D A T A   M E M O R Y   * * * * * * *
            REG     0000H     0008H     ABSOLUTE     "REG BANK 0"
            IDATA   0008H     0001H     UNIT         ?STACK

            * * * * * * *   C O D E   M E M O R Y   * * * * * * *
            CODE    0000H     0003H     ABSOLUTE     
            CODE    0003H     0012H     UNIT         ?PR?_DELAY?穇送文件
            CODE    0015H     0012H     UNIT         ?PR?INIT?穇送文件
            CODE    0027H     000DH     UNIT         ?PR?MAIN?穇送文件
            CODE    0034H     000CH     UNIT         ?C_C51STARTUP
            CODE    0040H     0009H     UNIT         ?PR?SEND?穇送文件



OVERLAY MAP OF MODULE:   485_Send (?C_STARTUP)


SEGMENT
  +--> CALLED SEGMENT
---------------------
?C_C51STARTUP
  +--> ?PR?MAIN?穇送文件

?PR?MAIN?穇送文件
  +--> ?PR?INIT?穇送文件
  +--> ?PR?SEND?穇送文件
  +--> ?PR?_DELAY?穇送文件



SYMBOL TABLE OF MODULE:  485_Send (?C_STARTUP)

  VALUE           TYPE          NAME
  ----------------------------------

  -------         MODULE        ?C_STARTUP
  C:0034H         SEGMENT       ?C_C51STARTUP
  I:0008H         SEGMENT       ?STACK
  C:0000H         PUBLIC        ?C_STARTUP
  D:00E0H         SYMBOL        ACC
BL51 BANKED LINKER/LOCATER V5.11                                                      02/09/2014  15:07:21  PAGE 2


  D:00F0H         SYMBOL        B
  D:0083H         SYMBOL        DPH
  D:0082H         SYMBOL        DPL
  N:0000H         SYMBOL        IBPSTACK
  N:0100H         SYMBOL        IBPSTACKTOP
  N:0080H         SYMBOL        IDATALEN
  C:0037H         SYMBOL        IDATALOOP
  N:0000H         SYMBOL        PBPSTACK
  N:0000H         SYMBOL        PBPSTACKTOP
  N:0000H         SYMBOL        PDATALEN
  N:0000H         SYMBOL        PDATASTART
  N:0000H         SYMBOL        PPAGE
  N:0000H         SYMBOL        PPAGEENABLE
  D:00A0H         SYMBOL        PPAGE_SFR
  D:0081H         SYMBOL        SP
  C:0034H         SYMBOL        STARTUP1
  N:0000H         SYMBOL        XBPSTACK
  N:0000H         SYMBOL        XBPSTACKTOP
  N:0000H         SYMBOL        XDATALEN
  N:0000H         SYMBOL        XDATASTART
  C:0000H         LINE#         92
  C:0034H         LINE#         99
  C:0036H         LINE#         100
  C:0037H         LINE#         101
  C:0038H         LINE#         102
  C:003AH         LINE#         151
  C:003DH         LINE#         155
  -------         ENDMOD        ?C_STARTUP

  -------         MODULE        穇送文件
  C:0000H         SYMBOL        _ICE_DUMMY_
  D:0080H         PUBLIC        P0
  B:0098H.1       PUBLIC        TI
  C:0027H         PUBLIC        main
  C:0040H         PUBLIC        send
  D:0099H         PUBLIC        SBUF
  D:0087H         PUBLIC        PCON
  D:0098H         PUBLIC        SCON
  D:0089H         PUBLIC        TMOD
  C:0015H         PUBLIC        init
  D:008DH         PUBLIC        TH1
  D:008BH         PUBLIC        TL1
  B:0088H.6       PUBLIC        TR1
  C:0003H         PUBLIC        _delay
  -------         PROC          _DELAY
  D:0007H         SYMBOL        k
  -------         DO            
  D:0006H         SYMBOL        j
  -------         ENDDO         
  C:0003H         LINE#         22
  C:0003H         LINE#         23
  C:0003H         LINE#         25
  C:0009H         LINE#         26
  C:0009H         LINE#         27
  C:0011H         LINE#         28
  C:0014H         LINE#         29
  C:0014H         LINE#         30
BL51 BANKED LINKER/LOCATER V5.11                                                      02/09/2014  15:07:21  PAGE 3


  -------         ENDPROC       _DELAY
  -------         PROC          INIT
  C:0015H         LINE#         41
  C:0015H         LINE#         42
  C:0015H         LINE#         43
  C:0018H         LINE#         44
  C:001BH         LINE#         45
  C:001EH         LINE#         46
  C:0021H         LINE#         47
  C:0023H         LINE#         48
  C:0026H         LINE#         49
  -------         ENDPROC       INIT
  -------         PROC          SEND
  C:0040H         LINE#         60
  C:0040H         LINE#         61
  C:0040H         LINE#         62
  C:0043H         LINE#         63
  C:0046H         LINE#         64
  C:0046H         LINE#         66
  C:0046H         LINE#         67
  C:0048H         LINE#         69
  -------         ENDPROC       SEND
  -------         PROC          MAIN
  C:0027H         LINE#         80
  C:0027H         LINE#         81
  C:0027H         LINE#         83
  C:002AH         LINE#         85
  C:002AH         LINE#         86
  C:002AH         LINE#         87
  C:002DH         LINE#         88
  C:0032H         LINE#         90
  -------         ENDPROC       MAIN
  -------         ENDMOD        穇送文件

Program Size: data=9.0 xdata=0 code=73
LINK/LOCATE RUN COMPLETE.  0 WARNING(S),  0 ERROR(S)
